:100000000EC026C025C024C023C022C021C020C0ED
:100010001FC01EC01DC01CC01BC01AC019C01124A7
:100020001FBECFEDCDBF10E0A0E6B0E0EAECF0E0FF
:1000300002C005900D92A036B107D9F710E0A0E6F6
:10004000B0E001C01D92A036B107E1F729D03BC056
:10005000D7CF82E087BD07B400FEFDCF87B58460AF
:1000600087BD82E087BB1EBC8FEF8DBD83E780BF5D
:1000700084E084BB81E287B980E886B90895369A26
:100080003699FECF85B10895982F8754883B10F498
:10009000965404C0973410F41EBC08959EBD089574
:1000A000F894D7DF7894369A3699FECF95B1892F98
:1000B0008754883B10F4965404C0973410F41EBC47
:0A00C000F2CF9EBDF0CFF894FFCF01
:00000001FF
